:040000004FEF00F0CE
:10000800FFFFFACF01F0FBCF02F0E9CF03F0EACF10
:1000180004F0E1CF05F0E2CF06F0D9CF07F0DACF50
:1000280008F0F3CF09F0F4CF0AF0F6CF0BF0F7CFD2
:100038000CF0F8CF0DF0F5CF0EF0F2949EAA01D097
:1000480001D007D002D001D000D0AECFADFF9E9A2C
:1000580000D0830ED626000ED7220EC0F5FF0DC0A5
:10006800F8FF0CC0F7FF0BC0F6FF0AC0F4FF09C089
:10007800F3FF08C0DAFF07C0D9FF06C0E2FF05C0DA
:10008800E1FF04C0EAFF03C0E9FF02C0FBFF01C0B3
:0A009800FAFF1100FFFF6AEF03F00A
:100600006C6B656D62656464656420626C756574AD
:100610006F6F74682074657374200D0A0000FFFF0B
:100620000F0E926E010E936E000E816E800E946E10
:10063000000E826E000E956E000E836E000E966E9A
:10064000000E846E440ED56EA40EF26E000ED76EB0
:10065000830ED66E200EAC6E900EAB6E190EAF6E82
:10066000200E9D6EE40EF26E1200FFFFFFFF000EE3
:10067000136E120E126E05D014C00FF060EC03F072
:1006800000D010C0F6FF11C0F7FF104A112A080071
:10069000FFFFF5CF14F0146601D001D0EDD700D0E4
:1006A0001200FFFFFFFF0FEC03F000D0060E116EEB
:1006B000000E106E36EC03F0F9D7F8D74FEF00F0CC
:1006C000FFFF00D0ACA201D001D0FCD70FC0ADFF1E
:1006D0001200FFFF000EF86E060EF76E000152EFDB
:0206E00003F025
:00000001FF
